:06000000020033020801BA
:03000B00020802E6
:03001300020803DD
:03001B00020804D4
:03002300020805CB
:03002B00020806C2
:10003300759840758780758921758DFF758BFF7560
:100043008840D299758107753001757700757800FE
:100053007533007531007535FFD210D211D212D22B
:1000630013D214D215D216D217D218D219D21AD249
:100073001BD21CD21DD21ED21FD234D235D236D2BD
:1000830037D240D241D242D243D244D245D246D2D1
:1000930047D248D249D24AD24BD24CD24DD24E1239
:1000A30013EF741FB535037535FF0535E535A2E04C
:1000B30092A4A2E192A5A2E292A6A2E392A7A2E44D
:1000C30092A1B392A2D2A3C2B0D29020901C753257
:1000D300031208F0120807D532067532011208F030
:1000E30012080ED29020900280EDC2A3D2912091EB
:1000F3001C753203120902120807D5320675320144
:1001030012090212080ED29120910280EDD29220A0
:100113009214301421C214B215201505120914804B
:1001230015120914801020140DD214201505120A7B
:10013300028003120A02D293209314301621C216AE
:10014300B217201705120A068015120A53801020D1
:10015300160DD216201705120A4F8003120A81D2F8
:1001630094209414301821C218B219201905120AC8
:10017300858015120A85801020180DD218201905C4
:10018300120C1C8003120C1CD295209514301A21DA
:10019300C21AB21B201B05120C208015120C4880BA
:1001A30010201A0DD21A201B05120C448003120CC6
:1001B3006CD296209614301C21C21CB21D201D0542
:1001C300120C708015120C988010201C0DD21C206C
:1001D3001D05120C948003120CBCD2972097143087
:1001E3001E21C21EB21F201F05120CC08015120C47
:1001F300E88010201E0DD21E201F05120CE4800380
:10020300120D0CD2B220B214303421C234B23520D4
:100213003505120D108015120D48801020340DD2B3
:1002230034203505120D448003120D70D2B320B370
:1002330014303621C236B237203705120D748015BB
:10024300120D74801020360DD236203705120DDBC7
:100253008003120DDBD2B420B414303821C238B27B
:1002630039203905120DDF8015120DDF801020387B
:100273000DD238203905120E298003120E29D2B56A
:1002830020B514303A21C23AB23B203B05120E2D61
:100293008015120E558010203A0DD23A203B0512DC
:1002A3000E518003120E79D2B620B614303C21C20F
:1002B3003CB23D203D05120E7D8015120EB080101C
:1002C300203C0DD23C203D05120EAC8003120ED60D
:1002D300D2B720B714303E21C23EB23F203F0512B1
:1002E3000EDA8015120F0E8010203E0DD23E203FF5
:1002F30005120F0A8003120F3ED2B0A2409290A2C1
:10030300419291A2429292A2439293A2449294A2C6
:10031300459295A2469296A2479297A24892A0A28E
:100323004992B2A24A92B3A24B92B4A24C92B5A202
:100333004D92B6A24E92B7E4B5350261FC04B535D1
:1003430002811C04B53502813C04B53502815C048D
:10035300B53502817C04B53502819C04B535028133
:10036300BC04B5350281DC04B5350281FC04B53526
:1003730002A11C04B53502A13C04B53502A15C04FD
:10038300B53502A17C04B53502A19C04B53502A1A3
:10039300BC04B53502A1DC04B53502A1FC04B535B6
:1003A30002C11C04B53502C13C04B53502C15C046D
:1003B300B53502C17C04B53502C19C04B53502C113
:1003C300BC04B53502C1DC04B53502C1FC04B53546
:1003D30002E11C04B53502E13C04B53502E15C04DD
:1003E300B53502E17C04B53502E19C04B53502E183
:1003F300BC04B53502E1DCE1FCE580F536A837A99C
:1004030036120815400624FE500D800512081A50B6
:1004130006853637120F42E1FCE580F538A839A985
:1004230038120815400624FE500D800512081A5094
:1004330006853839120F63E1FCE580F53AA83BA93C
:100443003A120815400624FE500D800512081A5072
:1004530006853A3B120F84E1FCE580F53CA83DA9F3
:100463003C120815400624FE500D800512081A5050
:1004730006853C3D120FA5E1FCE580F53EA83FA9AA
:100483003E120815400624FE500D800512081A502E
:1004930006853E3F120FC6E1FCE580F540A841A961
:1004A30040120815400624FE500D800512081A500C
:1004B30006854041120FE7E1FCE580F542A843A918
:1004C30042120815400624FE500D800512081A50EA
:1004D3000685424312100AE1FCE580F544A845A9CC
:1004E30044120815400624FE500D800512081A50C8
:1004F3000685444512102BE1FCE580F546A847A983
:1005030046120815400624FE500D800512081A50A5
:100513000685464712104CE1FCE580F548A849A939
:1005230048120815400624FE500D800512081A5083
:100533000685484912106DE1FCE580F54AA84BA9F0
:100543004A120815400624FE500D800512081A5061
:1005530006854A4B12108EE1FCE580F54CA84DA9A7
:100563004C120815400624FE500D800512081A503F
:1005730006854C4D1210B1E1FCE580F54EA84FA95C
:100583004E120815400624FE500D800512081A501D
:1005930006854E4F1210D2E1FCE580F550A851A913
:1005A30050120815400624FE500D800512081A50FB
:1005B300068550511210F3E1FCE580F552A853A9CA
:1005C30052120815400624FE500D800512081A50D9
:1005D30006855253121114E1FCE580F554A855A980
:1005E30054120815400624FE500D800512081A50B7
:1005F30006855455121137E1FCE580F556A857A935
:1006030056120815400624FE500D800512081A5094
:100613000685565712115AE1FCE580F558A859A9E9
:1006230058120815400624FE500D800512081A5072
:100633000685585912117BE1FCE580F55AA85BA9A0
:100643005A120815400624FE500D800512081A5050
:1006530006855A5B12119CE1FCE580F55CA85DA957
:100663005C120815400624FE500D800512081A502E
:1006730006855C5D1211BDE1FCE580F55EA85FA90E
:100683005E120815400624FE500D800512081A500C
:1006930006855E5F1211DEE1FCE580F560A861A9C5
:1006A30060120815400624FE500D800512081A50EA
:1006B30006856061121201E1FCE580F562A863A979
:1006C30062120815400624FE500D800512081A50C8
:1006D30006856263121224E1FCE580F564A865A92E
:1006E30064120815400624FE500D800512081A50A6
:1006F30006856465121247E1FCE580F566A867A9E3
:1007030066120815400624FE500D800512081A5083
:100713000685666712126AE1FCE580F568A869A997
:1007230068120815400624FE500D800512081A5061
:100733000685686912128BE1FCE580F56AA86BA94E
:100743006A120815400624FE500D800512081A503F
:1007530006856A6B1212AFE1FCE580F56CA86DA902
:100763006C120815400624FE500D800512081A501D
:1007730006856C6D1212D0E1FCE580F56EA86FA9B9
:100783006E120815400624FE500D800512081A50FB
:1007930006856E6F1212F1E1FCE580F570A871A970
:1007A30070120815400624FE500D800512081A50D9
:1007B3000685707112132AE1FCE580F572A873A90E
:1007C30072120815400624FE500D800512081A50B7
:1007D30006857273121363E1FCE580F574A875A9AD
:1007E30074120815400624FE500D800512081A5095
:1007F3000685747512139BE1FC01A50200333232A6
:10080300323232327E20DFFEDEFC227E60DFFEDE0D
:10081300FC22C2D7E89922C2D7E99824FE22309954
:10082300FDC299223099FDC2997599F03099FDC2A4
:10083300997599413099FDC2997599003099FDC216
:10084300997599003099FDC2997599233099FDC224
:10085300997599123099FDC2997599203099FDC205
:1008630099759901223099FDC2997599F03099FDD6
:10087300C2997599413099FDC2997599003099FDD6
:10088300C2997599003099FDC2997599233099FDE4
:10089300C2997599123099FDC2997599203099FDC5
:1008A300C299759902223099FDC2997599F722E58B
:1008B3007675F08084748095F020D201E43099FD40
:1008C300C299F5993099FDC2997599F722F5F0C44B
:1008D300540F3099FDC299F5992576F576E5F054D4
:1008E3000F3099FDC299F5992576F57622120821E4
:1008F3007599C01531E531547F120821F5992212FB
:1009030008217599C00531E531547F120821F59905
:1009130022120868120821759934E53304F533125D
:100923000821B40806E4F533020968B40103020997
:100933007EB40203020994B403030209AAB40403B4
:100943000209C0B405030209D6B406030209EC7513
:10095300990412082175990B12082175991B120825
:10096300A91208072275990112082175990912081D
:10097300217599201208A9120807227599021208F5
:10098300217599001208217599281208A9120807E0
:100993002275990212082175990512082175992368
:1009A3001208A91208072275990212082175990ADB
:1009B30012082175991E1208A912080722759903B6
:1009C30012082175990912082175991E1208A91296
:1009D30008072275990312082175990E12082175CB
:1009E30099191208A912080722759904120821758A
:1009F30099031208217599231208A91208072212D4
:100A0300080722E578B40004C244801EB40104C27E
:100A1300438017B40204C2408010B40304C241806F
:100A230009B40404C2428002C248120827120821F2
:100A330075997C1208217599001208217599011284
:100A430008217599621208A91208072212080722C1
:100A5300D244D243D240D241D242D24812082712C2
:100A6300082175997C12082175990012082175993E
:100A7300001208217599631208A9120807221208A7
:100A8300072230441130430E30400B3041083042CE
:100A930005304802811CE57804F578B40606E4F5D0
:100AA30078020AE9B40103020B31B40203020B79A1
:100AB300B40303020BC1B40403020BEBD244D243CD
:100AC300D240D241D242C248120827120821759956
:100AD3007E12082175990012082175990A120821BE
:100AE300759957020C15C244D243D240D241D24227
:100AF300D24812082712082175997E120821759988
:100B03000012082175990212082175995F1208A92C
:100B130012086812082175990412082175990012A8
:100B2300082175990012082175995A020C15D244AF
:100B3300C243D240D241D242D248120827120821DE
:100B430075997E1208217599001208217599021270
:100B5300082175995F1208A912086812082175996E
:100B630004120821759900120821759902120821AF
:100B7300759958020C15D244D243C240D241D24295
:100B8300D24812082712082175997E1208217599F7
:100B93000012082175990212082175995F1208A99C
:100BA3001208681208217599041208217599001218
:100BB3000821759903120821759957020C15D2441F
:100BC300D243D240C241D242D2481208271208214E
:100BD30075997E12082175990012082175990112E1
:100BE3000821759960020C15D244D243D240D241F8
:100BF300C242D24812082712082175997E12082191
:100C030075990012082175990712082175995A02DE
:100C13000C151208A91208072212080722C245124E
:100C230008271208217599241208217599001208C2
:100C33002175990112082175993A1208A91208071A
:100C43002212080722D24512082712082175992477
:100C5300120821759900120821759900120821754F
:100C6300993B1208A91208072212080722C246124A
:100C73000827120821759960120821759900120836
:100C83002175990112082175997E1208A912080786
:100C93002212080722D246120827120821759960EA
:100CA30012082175990012082175990012082175FF
:100CB300997F1208A91208072212080722C24712B5
:100CC300086812082175993C1208217599001208C9
:100CD300217599011208217599211208A912080793
:100CE3002212080722D24712086812082175993C7C
:100CF30012082175990012082175990012082175AF
:100D030099221208A91208072212080722E530B413
:100D13000004C24A8009B40104C2498002C24B12D2
:100D2300086812082175994C120821759900120858
:100D3300217599011208217599111208A912080742
:100D43002212080722D24AD249D24B12086812084B
:100D53002175994C12082175990012082175990083
:100D63001208217599121208A912080722120807FE
:100D730022304A08304905304B02805C1208681261
:100D8300082175994E120821759900E53004F53054
:100D9300120821B40305E4F5308025B40111D24AC9
:100DA300C249D24B75990212082175990E8022D23D
:100DB3004AD249C24B75990412082175990C8011C6
:100DC300C24AD249D24B75990012082175991080F5
:100DD300001208A912080722120807221208271274
:100DE3000821759956120821759900E57704F5775E
:100DF300120821B40305E4F5778019B4010B759942
:100E03000112082175990880167599021208217537
:100E13009907800B759900120821759909800012B2
:100E230008A91208072212080722C24C1208271227
:100E330008217599441208217599001208217599A2
:100E43000112082175991A1208A91208072212081B
:100E53000722D24C1208271208217599441208213F
:100E630075990012082175990012082175991B12B2
:100E730008A91208072212080722204F06D24EC2E1
:100E83004D8004C24ED24D12086812082175992C68
:100E9300120821759900120821759901120821750C
:100EA30099311208A91208072212080722D24ED23A
:100EB3004D12086812082175992C120821759900A2
:100EC3001208217599001208217599321208A91286
:100ED30008072212080722304E05304D028028C22F
:100EE3004DD24EC24F12086812082175992E12086E
:100EF3002175990012082175990112082175992FFE
:100F03001208A91208072212080722304E05304D95
:100F1300028028D24DC24ED24F12086812082175A2
:100F2300992E12082175990012082175990012084B
:100F3300217599301208A9120807221208072212F4
:100F4300082712082175994E75766FE53694C850B7
:100F530004E536800274C8C3131208D01208B22203
:100F630012082712082175994C75766DE53894C8D7
:100F73005004E538800274C8C3131208D01208B2B3
:100F83002212082712082175994A75766BE53A945F
:100F9300C85004E53A800274C8C3131208D012087B
:100FA300B222120827120821759950757671E53C13
:100FB30094C85004E53C800274C8C3131208D012CD
:100FC30008B222120827120821759948757669E537
:100FD3003E94C85004E53E800274C8C3131208D07F
:100FE3001208B222120827120821759946757667EE
:100FF300E54094CC5004E540800274CC75F00C8439
:101003001208D01208B22212086812082175993A00
:1010130075765CE54294C85004E542800274C8C307
:10102300131208D01208B222120868120821759907
:1010330030757652E54494B45004E544800274B4A8
:10104300C3131208D01208B22212086812082175BD
:101053009936757658E54694C85004E5468002747F
:10106300C8C3131208D01208B2221208681208214A
:10107300759934757656E54894C85004E54880025E
:1010830074C8C3131208D01208B2221208681208D7
:101093002175993875765AE54A94DC5004E54A80FF
:1010A3000274DC75F014841208D01208B2221208FC
:1010B3006812082175995A75767CE54C94C85004DA
:1010C300E54C800274C8C3131208D01208B222126E
:1010D3000868120821759950757672E54E94C850C8
:1010E30004E54E800274C8C3131208D01208B2225A
:1010F300120868120821759952757674E55094C8E0
:101103005004E550800274C8C3131208D01208B209
:101113002212086812082175995875767AE5529457
:10112300DC5004E552800274DC75F014841208D09C
:101133001208B2221208681208217599567576783A
:10114300E55494DC5004E554800274DC75F0148497
:101153001208D01208B222120868120821759940A9
:10116300757662E55694C85004E556800274C8C388
:10117300131208D01208B2221208681208217599B6
:101183004875766AE55894C85004E558800274C8D7
:10119300C3131208D01208B22212082712082175AD
:1011A3009952757673E55A94C85004E55A800274CF
:1011B300C8C3131208D01208B222120868120821F9
:1011C300759942757664E55C94C85004E55C8002C9
:1011D30074C8C3131208D01208B2221208271208C7
:1011E30021759962757683E55E94C85004E55E8047
:1011F3000274C875F005841208D01208B2221208CE
:1012030027120821759968757689E56094C850049A
:10121300E560800274C875F005841208D01208B224
:101223002212082712082175996E75768FE562944C
:10123300C85004E562800274C875F005841208D0B2
:101243001208B22212082712082175997075769137
:10125300E56494C85004E564800274C875F005849D
:101263001208D01208B22212082712082175992EEB
:1012730075764FE56694C85004E566800274C8C36A
:10128300131208D01208B2221208271208217599E6
:101293002A75764BE56894C85004E568800274C8E3
:1012A300F49436C3131208D01208B222120827127C
:1012B3000821759928757649E56A94C85004E56A4A
:1012C300800274C8C3131208D01208B2221208276E
:1012D300120821759976757697E56C94C85004E5E4
:1012E3006C800274C8C3131208D01208B222120809
:1012F30068E578120821B403087599047576268089
:1013030011B40408759904757626800675990675D7
:101313007628E56E94C85004E56E800274C8C31342
:101323001208D01208B222120868E578120821B414
:1013330003087599067576288011B4040875990613
:10134300757628800675990875762AE57094C850D5
:1013530004E570800274C8C3131208D01208B222C5
:10136300E578B4040122B4050122120868E5781275
:101373000821B4030875990A75762C800675990CB3
:1013830075762EE57294C85004E572800274C8C362
:10139300131208D01208B222E578B404012212080D
:1013A30068E578120821B4030875990875762A80D0
:1013B30026B4051D759904757626E57494DC5004EE
:1013C300E574800274DC75F00B841208D01208B245
:1013D3002275990A75762CE57494C85004E57480D7
:1013E3000274C8C3131208D01208B222C29412089E
:1013F30007C293120807C290120807C29112080786
:10140300C292120807C2A0120807C295C296C297D9
:10141300C2B5C2B3C2B2C2B4C2B6C2B712080712CF
:101423000807120807D295D296D297D2B5D2B3D273
:10143300B2D2B4D2B6D2B7120807120807120807FD
:10144300C295C296C297C2B5C2B3C2B2C2B4C2B643
:10145300C2B7120807120807120807D295D296D20C
:1014630097D2B5D2B3D2B2D2B4D2B6D2B71208079A
:10147300120807120807C295C296C297C2B5C2B333
:10148300C2B2C2B4C2B6C2B7120807120807120822
:1014930007D295D296D297D2B5D2B3D2B2D2B4D222
:1014A300B6D2B7120807120807120807D2A012080B
:1014B30007D292120807D291120807D29012080796
:1014C300D293120807D29412080722204D757A7915
:1014D3006B616E7420382076312E306120323030CB
:1014E300372D31322D3135202863294164616D2038
:1014F300536D69616C656B206A616E6B6F6D757A94
:10150300796B616E744077702E706C207777772ECD
:10151300736D69616C656B2E7072762E706C2057DB
:10152300737A656C6B6965207072617761207A618B
:101533007374727A657A6F6E652E204A616B696582
:101543006B6F6C7769656B207A6173746F736F77F8
:10155300616E6961206B6F6D657263796A6E652078
:101563006B6F6475206E6965646F7A776F6C6F6EED
:10157300652E20416C6C2052696768747320526534
:101583007365727665642E204672656520666F7298
:10159300206E6F6E20636F6D6D65726369616C2081
:0615A3006F6E6C792E2032
:00000001FF
